:100000008C282A20A0000408A200080090002208E2
:1000100084002008272084130005181C20060319DB
:1000200024281008031D1C281608FF3E031C252841
:100030000A303C2016082528100AFF30031924280E
:10004000100B2428170825289909990C872884174C
:10005000800487289400063094190530840000300D
:100060008A00140807398207013402340434083442
:1000700010342034403480348F018E00FF308E07DE
:10008000031C8F07031C872803308D00DF304A20B4
:100090003E288D01E83E8C008D09FC30031C53285E
:1000A0008C07031850288C0764008D0F50280C18FB
:1000B00059288C1C5D2800005D28080093019200DF
:1000C0001C308E006F308F0071200F30831681043A
:1000D0008312FF3063008C07031C8D0703186A2806
:1000E0008728103094008D018C01930C920C031C16
:1000F0007F280E088C070F0803180F0F8D078D0C33
:100100008C0C910C900C940B752810088728831385
:100110000313831264000800A701A401A501A6012E
:1001200013308F0088303D20831680308600831284
:100130000130A70064000C3027020318A228D42045
:10014000A70F9A28073001209801FF3096009701E9
:100150000130990026080620A6000318CF28023097
:10016000930058305F200130A70064000C30270254
:100170000318BD28ED20A70FB5280610831606101A
:1001800083128610831686108312061183160611B9
:10019000831286118316861163008312CC280730E0
:1001A000930008305F20B3280C30860013308F0096
:1001B00088303D200630860013308F0088303D2087
:1001C0000330860013308F0088303D2009308600D0
:1001D00013308F0088303D2008000930860013302E
:1001E0008F0088303D200330860013308F00883028
:1001F0003D200630860013308F0088303D200C30C3
:0C020000860013308F0088303D2008007D
:02400E00F53F7C
:00000001FF
